:0600000006C05AC053C106
:02000800D7C05F
:10000C00C5C08FED8DBF88278BBD84EB8ABD85E085
:10001C0083BFA8958AE081BD80E888B980E087BB62
:10002C008FEF88BB81E281BB8FEF82BB80E085BF05
:10003C0080EC8BBF82E489BF78947727AA27A3959D
:10004C00A43669F1123071F1BE9907C0B6991BC084
:10005C0088278BBF1127C398BB9ABF9904C0B79947
:10006C0015C0C498BC9ABB9907C0B39912C0882715
:10007C008BBF1127C698BE9ABC99E1CFB4990CC01E
:10008C00C798BF9ADCCFBB98C39AE7CFBC98C49AE9
:10009C00EACFBE98C69AF0CFBF98C79AD0CFA89592
:1000AC00AA27D2CF80EC8BBF13E0CECF0FB6AA27F6
:1000BC0088278BBF789481E083BF1127D72F71607D
:1000CC00113150F5829BFCCF812F1127182E1694DD
:1000DC00212C180E880F280E1115F0F48299FCCFE4
:1000EC0011270CE0332722271115F0F3829909C050
:1000FC008894331F221F121578F4829BFCCF112792
:10010C0008C00894331F221F121530F48299FCCFBB
:10011C0011270A9549F701C031C0832F881F221F70
:10012C00881F221F25FB36F93F732F7190E282B393
:10013C00892782BB72FF02C0D4D020C021D14030AD
:10014C00E9F05030B9F0403E59F0342F72D0352FD1
:10015C0070D072D0342F6DD06FD0352F6AD00EC0C6
:10016C00342F67D0352F65D0342F63D065D0352F21
:10017C0060D004C0342F5DD05FD05BD07D2F85E084
:10018C0083BF8FEF8ABF8BBF0FBE18950FB6139529
:10019C006A9570FD09C0C395C83009F005C0CC271D
:1001AC0091E082B3892782BB0FBE18950FB6B39B23
:1001BC0002C039D019C03AD064E01DD0083051F0DB
:1001CC00093069F00A3069F0979510F026D00BC011
:1001DC0027D009C016F424D006C01FD004C020D0EC
:1001EC0002C07D7F01C003950FBE1895A8956030A5
:1001FC0009F0FCCF0895603079F000000000000099
:10020C0000000000000000000000000000000000E2
:10021C00000000006A95EFCF0895C498BC9A089529
:10022C00BC98C49A0895C398BB9A0895BB98C39A76
:10023C0008951FD0932F02C090EF6894726000272E
:10024C00B39B16C0B49B14C0E8DF64E0D4DFEBDFD3
:10025C0089E08EBD71FDFECF82E089BF88278EBDFF
:10026C0088278DBD88278CBD82E489BF64E1BEDF01
:10027C000895932F002788278894083029F0991F18
:10028C0008F483950395F9CF813041F0833031F038
:10029C00853021F0873011F068940895E894089522
:1002AC000FB688278BBF81E083BF78946EE49EDF06
:1002BC0083990FC084E0782772FD02C07E7F02C054
:1002CC0071609098A895839BFDCF6EE48FDF839B24
:1002DC00F9CF85E083BF8FEF8ABF80EC8BBF0FBE59
:1002EC001895E199FECFB1E0A895B799FDCF4427B9
:1002FC000027B699FECFB69BFECFB699FECFB79B23
:10030C0003C00894479502C088944795039508301C
:10031C0011F01127F0CF3F93342FABDF3F91B69BF9
:10032C00FECFB699FECFB79B02C02EF001C01EF4D3
:10033C0065E05CDF0895B23039F0542F330F19D0DB
:10034C0065E054DFB395D0CF90E282B3892782BBAE
:10035C00403F69F0451759F0E199FECF339509D02C
:10036C0084E083BF6CE042DF81E083BF08954427C3
:10037C00F3CF3EBB4DBBF894E29AE19A7894089582
:10038C00E199FECF330F3EBBE09A4DB3E199FECF1E
:0A039C0033953EBBE09A5DB308956F
:00000001FF
